:100000000C9462000C94C61A0C94F31A0C948A0097
:100010000C948A000C948A000C948A000C948A0038
:100020000C948A000C948A000C948A000C948A0028
:100030000C948A000C94900B0C948A000C948A0007
:100040000C94201B0C948A000C949C1E0C94DF1EB4
:100050000C948A000C948A000C948A000C948A00F8
:100060000C94F1080C948A000000000700020100C3
:100070000003040600000000000000000102040864
:100080001020408001020408102001020408102002
:10009000040404040404040402020202020203032E
:1000A00003030303000000002300260029000000D2
:1000B0000000250028002B0000000000240027007D
:1000C0002A00532011241FBECFEFD8E0DEBFCDBFE2
:1000D00012E0A0E0B1E0EAE1F3E402C005900D9285
:1000E000A23DB107D9F714E0A2EDB2E001C01D9224
:1000F000AC3BB107E1F710E0C4ECD0E004C02297BC
:10010000FE010E946821C23CD107C9F70E948F20DE
:100110000C948B210C9400008091BE03813019F463
:1001200082E08093BE038091BE03833019F484E0A3
:100130008093BE030895A8950895CF93DF93FC01A3
:10014000962F9270862F817060FF20C0992331F026
:100150008091500380831092D20216C0A091D202E7
:10016000C091E903C770D0E0C656DD4F8881A8175B
:1001700010F080E03CC081E08A0F8093D202B0E0B2
:10018000A050BD4F8C91808381E031C09923C1F094
:1001900090819093D3021092D202292F207E203694
:1001A00051F490915003923020F390819F7190937D
:1001B000920393E01AC09E3F39F71092500317C084
:1001C0009091D3029F3F01F79091D202993288F625
:1001D00021E0290F2093D2023081E92FF0E0EF5384
:1001E000FC4F3083293281F691E090935003DF91E8
:1001F000CF910895DC01ED91FC910190F081E02D0B
:1002000009950895DC01ED91FC910190F081E02DBC
:10021000099508952091BF033091C003382748E025
:10022000C901880F991F37FF06C09C0151E225279D
:1002300050E1352701C09C01415091F73093C00334
:100240002093BF0308958436910520F4BC0180E01B
:1002500090E017C09C018E3B910528F42A55310986
:10026000AAE0B0E00CC0823D910528F4245B31097E
:10027000A4E6B0E004C02D5C3109A8E5B2E00E941C
:100280009C20A4E6B0E09B01AC010E94AB20089545
:1002900090E08C599F4F0E942301089582E0809343
:1002A000EA0380E28093EB0386E28093EC0391E221
:1002B0009093ED038093EE0384E08093EF0385E059
:1002C0008093F00384E28093F10385E28093F2034C
:1002D000089560E08CE00E942E1C61E08BE00E949B
:1002E0002E1C61E08DE00E942E1C60E082E00E94E6
:1002F0002E1C61E084E00E942E1C089542E050E034
:100300006CE870E080E00E94A61A0895E3E0F0E057
:1003100089E080935700E491E67081E0E63009F0CF
:1003200080E00895CF93DF93C82F0E948601882331
:1003300081F0DFB781E08093BD03F8940E949B00B9
:1003400088E180936000C0936000C1110E949B000F
:10035000DFBFDF91CF910895FC0140A5842F877006
:1003600090E0959587950196242F217030E0820FBB
:10037000931F880F880F08958F929F92AF92BF921C
:10038000CF92DF92EF92FF92CF93FC01C0A5EC2FAA
:10039000E770F0E0E656FD4FA081B0E0C7FF03C074
:1003A00024E130E002C02FE030E0FC0197A183E1BE
:1003B000989FF0011124E25AFE4F80809180A28024
:1003C000B380A20FB31F20E43FE14DE750E00E944D
:1003D000B620A50194010E94EE208C2F887149F46B
:1003E00069017A01E0EDCE0EE7E0DE1EE11CF11CB2
:1003F0001BC0C7FF05C060E47AE88CE29EE004C041
:1004000060E07EEE8AEB9BE069017A01F8EBCF0EAB
:10041000FBE0DF1EE11CF11CA50194010E94EE200F
:10042000C20ED31EE41EF51EC701B60169517C4FF2
:100430008F4F9F4F28EE33E040E050E00E94EE20C7
:10044000A8EEB3E00E94AB20CF91FF90EF90DF9039
:10045000CF90BF90AF909F908F900895DB01FA01ED
:10046000582F569590E02481237030E0322F2227B8
:100470004081240F311D11963C932E9344814C7082
:10048000218130E060E4469F200D311D1124139638
:100490003C932E93129744814073228130E060E1B7
:1004A000469F200D311D112415963C932E931497D1
:1004B0004481407C238130E064E0469F200D311D63
:1004C000112417963C932E931697359618969F5F96
:1004D000591748F680FF47C040814295469546959A
:1004E00043702DE431E0429FC001439F900D1124E1
:1004F0000C9611969C938E93808190E074E0969573
:1005000087957A95E1F783709927829FA001839F51
:10051000500D929F500D1124445F5F4F13965C93D2
:100520004E931297808190E0969587959695879542
:1005300083709927829FA001839F500D929F500D39
:100540001124445F5F4F15965C934E93149740813E
:100550004370429FC001439F900D11240C96179643
:100560009C938E9316970895803223E0920708F1AA
:10057000883E23E0920740F48F519340E4E0969543
:100580008795EA95E1F70895803D27E0920718F4F2
:100590008C5D93400895883928E0920768F4885C60
:1005A000974074E0969587957A95E1F78D509C4F2A
:1005B000089580E090E008958FEF93E008958C30E7
:1005C000910540F4A4E0880F991FAA95E1F7885D92
:1005D0009C4F0895843F23E0920718F484529C4F67
:1005E0000895811524E0920740F48657934FF4E074
:1005F000880F991FFA95E1F7089580E998E008952A
:100600009C013695279525753575821B930B9C01AA
:100610002373337396958795969587958373937314
:10062000820F931F9C0154E0369527955A95E1F768
:10063000280F391F2F703F7041E051E0249FC00107
:10064000259F900D349F900D1124892F08952D988A
:10065000882319F000002B9A02C000002B9800009C
:100660002D9A000008952D9A000083B12D98000066
:10067000829581700895CF93DF93D82F5C9A2D983F
:100680005C98C8E08D2F80780E942703DD0FC15051
:10069000C9F72D98DF91CF9108958F770E943B0382
:1006A0000895CF93DF93D82FC8E08D2F80780E94D4
:1006B0002703DD0FC150C9F72D98DF91CF91089521
:1006C000CF93DF932D98C8E080E0D82FDD0F0E94F4
:1006D00033038D0FC150C9F7DF91CF9108950E9468
:1006E0004D030E9460035C9A0895A1E0B0E0EBE73F
:1006F000F3E00C943F21806869830E943B03698189
:10070000862F0E9451035C9A2196E2E00C945B21B3
:10071000CF93C091CA03C827E82FF0E0EF53FC4FF6
:10072000678589E70E9475036C2F8DE30E9475032E
:100730006C2F82E40E947503CF91089586E20E9497
:100740006F030895CF938BE20E946F03C82F8CE252
:100750000E946F03282F30E066E0369527956A9552
:10076000E1F744E0C49FC0011124822B932BCF9169
:100770000895CF93DF93EC016C818CE10E947503A7
:100780006D818DE10E9475036E818EE10E9475037B
:100790006F8180E20E947503688581E20E94750383
:1007A000698582E20E9475036A8583E20E9475036F
:1007B0006B8584E20E9475036C8585E20E94750357
:1007C0006D858AE20E9475036E858EE60E94750330
:1007D0006F858FE60E947503688980E70E94750324
:1007E000698981E70E9475036A8982E70E9475031F
:1007F000DF91CF910895CF92DF92EF92FF92CF9346
:10080000DF936B017C01C11488E3D8068CE9E8060C
:100810008CE1F80628F5C701B60120E836E948E979
:1008200050E00E94EE20E901689760E879E687E6EB
:100830009FEF0E94BE206C0D7D1D8E1D9F1DF2E05E
:10084000660F771F881F991FFA95D1F721E732E0CD
:1008500040E050E00E94EE20F22EE32E80E421C022
:10086000C701B60120E03DE241E351E00E94EE20E5
:10087000E901689760E073ED8EEC9EEF0E94BE2068
:100880006C0D7D1D8E1D9F1D660F771F881F991F84
:1008900021E732E040E050E00E94EE20F22EE32E0D
:1008A00080E66C2F6F71680F85E70E9475036E2DCF
:1008B00086E70E9475036F2D87E70E947503DF911D
:1008C000CF91FF90EF90DF90CF9008958F929F92FD
:1008D000AF92BF92CF92DF92EF92FF92CF93DF93CE
:1008E000D82F83E00E946F038093BC0384E00E94B2
:1008F0006F038093BB0360E086E00E94750361E0B4
:1009000087E00E9475036FE789E00E94750365E048
:100910008AE00E94750362E18BE00E94750365E145
:100920008CE00E9475036DEF8DE00E94750360E01E
:100930008EE00E947503DD2319F08BE491E008C07E
:100940002091E80333E1239FC0011124825A9E4F76
:100950000E94B9036CE880E30E9475036FE082E3B4
:100960000E94750362E483E30E9475038091E903AA
:1009700087FF02C064E101C06AE084E30E9475035E
:100980006AE285E30E9475036DE286E30E947503C7
:1009900064ED87E30E94750360E088E30E947503BD
:1009A00060E089E30E947503D11109C0C090CA03B9
:1009B000D090CB03E090CC03F090CD0307C0C5E905
:1009C000CC2EC1ECDC2EED2CCEEDFC2ECAE38F2C10
:1009D0009924AA24BB24682D8C2F0E947503682DAE
:1009E00085E08C0F0E947503FE2CED2CDC2CCC24B2
:1009F000CF5FCE3361F76FEF83E40E9475036FEF33
:100A000084E40E9475036FEF85E40E9475036FEF25
:100A100086E40E947503DD2311F066E002C0609158
:100A2000CE038DE60E94750360E089E70E9475039E
:100A30006091CF038AE70E94750360E083E70E941C
:100A4000750360E084E70E947503D11109C06091CD
:100A5000C6037091C7038091C8039091C90304C075
:100A600060EC72E98DEE99E10E94FB03DF91CF917A
:100A7000FF90EF90DF90CF90BF90AF909F908F90BE
:100A8000089561E087E00E94750364E28EE70E94AA
:100A9000750363E088E00E94750360E088E00E94CF
:100AA000750365E087E00E94750362E085E00E94BF
:100AB000750383E00E946F038093BC0384E00E946F
:100AC0006F038093BB03089583E00E946F038093BC
:100AD000BC0384E00E946F038093BB0361E087E066
:100AE0000E9475036AE070E080E090E00E94991B2C
:100AF0000E94410500000895CF92DF92FF920F936C
:100B00001F93CF93DF931F92CDB7DEB7082F162F19
:100B10008EE399830E947503F02EC02E9981D92E01
:100B20008C2D8F19811738F4F60161916F018FE7D1
:100B30000E947503F5CF64E085E00E94750383E0B1
:100B40000E946F038093BC0384E00E946F03809334
:100B5000BB030E94761B6093B7037093B803809326
:100B6000B9039093BA0369E087E00E94750381E0BE
:100B70008093BE030F90DF91CF911F910F91FF9053
:100B8000DF90CF9008950F931F930E947C05809172
:100B9000BE03813099F40E94761B0091B703109137
:100BA000B8032091B9033091BA03601B710B820B1B
:100BB000930B603A76488140910548F38091BE03DB
:100BC000813031F46EEB71E082E194E00E94381DD7
:100BD0001F910F9108950F931F938091BE03823050
:100BE00021F41092BE0381E020C08091BE038130C9
:100BF000D9F40E94761B0091B7031091B80320919D
:100C0000B9033091BA03601B710B820B930B613AED
:100C100076488140910540F061E087E00E947503CD
:100C20001092BE0382E001C080E01F910F910895F1
:100C3000EF92FF920F931F93CF93DF938B019C0151
:100C4000442737FD4095542F60E271EA87E090E039
:100C50000E941021E9011C161D0614F0C1E0D0E02D
:100C6000D80120E231EA47E050E00E94B6209E0120
:100C7000442737FD4095542F0E941021790100E050
:100C800010E00E151F055CF42B9ACE010E94BF1BCD
:100C90002B98CE010E94BF1B0F5F1F4FF2CFCDB725
:100CA000DEB7E6E00C945721CF93DF935D9A609115
:100CB000FA037091FB038091FC039091FD030E9465
:100CC000FB0360E089E70E94750361E070E080E06B
:100CD00090E00E94991B0E949E03C82F61E070E083
:100CE00080E090E00E94991B0E949E03D0E0C80F14
:100CF000D11D61E070E080E090E00E94991B0E94AD
:100D00009E03C80FD11D61E070E080E090E00E947A
:100D1000991B0E949E035D989E01280F311DC901F9
:100D20009695879596958795DF91CF910895CF9366
:100D3000C82F5D9A83E00E946F038093BC0384E018
:100D40000E946F038093BB0360E086E00E947503FE
:100D500061E087E00E9475036FE789E00E947503F8
:100D600065E08AE00E94750362E18BE00E947503F2
:100D700065E18CE00E9475036DEF8DE00E947503C4
:100D800060E08EE00E9475036CE280E70E947503CC
:100D900060E080E30E94750360E089E70E947503CC
:100DA00065E08AE70E94750362E181E70E947503AE
:100DB00062E082E70E94750360E083E70E947503AA
:100DC00060E084E70E9475036091FA037091FB0371
:100DD0008091FC039091FD030E94FB0367E08DE688
:100DE0000E9475036AE070E080E090E00E94991B29
:100DF00069E087E00E9475036AE070E080E090E0BF
:100E00000E94991BCC2369F0C5E1C15009F459C077
:100E100061E070E088EB91E00E9418060E949B0060
:100E2000F4CF61E070E088E891E00E9418060E942B
:100E30009B0065E08DE60E9475036AE070E080E04B
:100E400090E00E94991B61E070E088EB91E00E94C5
:100E500018060E949B0064E08DE60E9475036AE01C
:100E600070E080E090E00E94991B61E070E08DE509
:100E700091E00E9418060E949B0062E08DE60E94AD
:100E800075036AE070E080E090E00E94991B61E0E9
:100E900070E08FEA90E00E9418060E949B0060E0DC
:100EA0008DE60E9475036AE070E080E090E00E94A9
:100EB000991B62E070E085E091E00E9418060E94B4
:100EC0009B0061E087E00E9475035D98CF910895D3
:100ED000CF93DF93EC014AE050E06D2F70E082E1A8
:100EE00094E00E94FD1D6EE282E194E00E941C1DD0
:100EF000BE0184E0769567958A95E1F76F70772754
:100F00004AE050E082E194E00E94FD1D6EE282E141
:100F100094E00E941C1DBE016F7077274AE050E0EC
:100F200082E194E00E94FD1DDF91CF910895D82FBA
:100F3000C0E0CD1780F45E9A64E670E080E090E057
:100F40000E94991B5E9864E670E080E090E00E9449
:100F5000991BCF5FEECF6CE271E080E090E00E94E1
:100F6000991BE6CF0F931F93CF93DF93EC01062FCE
:100F700015E0115051F0CE010E947521081741F083
:100F8000602FCE010E947D21F4CF82E00E9497075E
:100F9000DF91CF911F910F910895A0E0B0E0E3EDB4
:100FA000F7E00C943121482E562EC0E0D0E0612CA1
:100FB000712CE12CF12C00E010E0442079F081E06C
:100FC0004816A1F092E0491219C028E4622E712C53
:100FD00030E2E32EF12C03E513E010C0612C712CFC
:100FE0006BE1E62EF12C0AEE13E008C04DE1642E11
:100FF000712C59E2E52EF12C01EC13E043018C0E2B
:101000009D1E1092C0031092BF033401A62CA81895
:10101000B12CC30101966C01AE14BF04A8F4A00E5C
:10102000B11E511006C0C3010E947521F5018083D5
:1010300005C0F5016081C3010E94B207F5018081FE
:101040000E940A013601E2CFC301511018C0C3014A
:101050000E947521B82EC6010E9475212B2D30E00B
:10106000322F2227282B8091BF039091C003821733
:10107000930779F4C0E0D0E0552453949ECF360115
:101080006091C0030E94B2076091BF03C6010E9435
:10109000B207D395C13093E0D90708F48ECF852DE0
:1010A000CDB7DEB7E0E10C944D2160E081E00E9415
:1010B000CD07882331F081E09091C103983309F086
:1010C00080E0089561E081E00E94CD07089561E02D
:1010D00082E00E94CD07089560E082E00E94CD0783
:1010E000811108C0E3E5F3E01192119283E0E33748
:1010F000F807D1F70895A1E0B0E0E1E8F8E00C943A
:101100003F2189830E944E0192E09093F8039FEF64
:101110009093F9039AE090930204109203041092C2
:1011200004041092FA031092FB031092FC03109235
:10113000FD032EE12093FE039093FF0328EB3BE099
:1011400030930104209300048981882371F061E0C9
:1011500080E00E94CD07E3E5F3E01192119283E075
:10116000E337F807D1F70E9467082196E2E00C9474
:101170005B2160E080E00E94CD07811103C081E027
:101180000E947B080895CF93C1E0811101C0C0E0A7
:101190006C2F82E10E94671C6C2F83E10E94671C08
:1011A0001092B1031092B0038091B9008C6F8093BC
:1011B000B90080E28093B80085E48093BC00CF91B1
:1011C000089585ED8093BC008091BC0084FDFCCF28
:1011D0000895ECEBF0E0108285E480831092B00378
:1011E00008951F920F920FB60F9211242F933F93E1
:1011F0004F935F936F937F938F939F93AF93BF931F
:10120000EF93FF93CF93DF931F92CDB7DEB780911B
:10121000B900887F803609F4C7C0A8F5883209F480
:1012200064C098F4803109F45DC038F4882309F46F
:10123000F3C0883009F456C0F1C0883109F455C0B4
:10124000803209F0EBC082E0A7C0803409F477C097
:1012500078F4803309F45FC0883309F0DFC084E09C
:101260008093AF038091B0038B7F8093B003D0C095
:10127000803509F452C0883509F467C0883409F014
:10128000CDC085E089C0883909F4C0C0A8F488378A
:1012900009F48AC038F4883609F486C0803709F426
:1012A00083C0BCC0883809F4B1C0803909F47FC05C
:1012B000803809F0B3C07BC0803B09F493C038F498
:1012C000803A09F48CC0883A09F48CC0A7C0803CED
:1012D00009F49EC0883C09F49BC0883B09F09EC07D
:1012E00080E081C08091B40313C08091B1039FEF6F
:1012F000980F9093B1038823D1F1E091B203F0915C
:10130000B303CF0101969093B3038093B20380811E
:101310008093BB007DC083E03FC0E091B203F091B9
:10132000B303CF0101969093B3038093B2038091EE
:10133000BB0080838091B10381508093B103809181
:10134000B103823008F064C061C0E091B203F09153
:10135000B303CF0101969093B3038093B2038091BE
:10136000BB0080838091B10381508093B103809151
:10137000B0038B7F8093B0038091B00380FF4CC09B
:101380008091B0038E7F8093B0038091B003826020
:101390008093B00384EA3DC08093AF038091B00393
:1013A0008B7F8093B00338C01092B10331C0E091BD
:1013B000B503F091B603309749F18091BB00898362
:1013C0008091B10391E0980F9093B103811102C015
:1013D00062E001C060E0CE010196099515C00E944F
:1013E000E10816C081E0E091B503F091B6033097B3
:1013F00069F0882311F063E001C061E0CE0101963D
:10140000099599819093BB00811102C085E801C0C4
:1014100085EC8093BC0002C00E94E1080F90DF9130
:10142000CF91FF91EF91BF91AF919F918F917F915C
:101430006F915F914F913F912F910F900FBE0F9041
:101440001F9018958F929F92AF92BF92CF92DF928A
:10145000EF92FF92CF93DF93EC010E94761B6B011A
:101460007C014E01A12CB12C8091B00382FF11C0F0
:101470002097D1F30E94761B6C197D098E099F0974
:1014800086169706A806B90678F70E94E90881E053
:1014900004C08091AF031092AF03DF91CF91FF9012
:1014A000EF90DF90CF90BF90AF909F908F90089576
:1014B000A2E0B0E0EEE5FAE00C943B21182F7B01AE
:1014C000022F047022FD05C080910B0190910C0148
:1014D00002C080E090E02A8349830E94220A2A8188
:1014E0004981811136C01092AF034093B103F0924D
:1014F000B303E092B203110F1093B4039091B003C1
:1015000021FF02C085E001C084E0892B8093B003F5
:101510008091B00381FF0BC08091B0038D7F8093D9
:10152000B0038091B4038093BB0085EC01C085EECD
:101530008093BC00822F817020FF0BC0011105C079
:1015400080910B0190910C0102C080E090E00E941C
:10155000220A2296E6E00C945721A2E0B0E0E3EBE9
:10156000FAE00C943B21182F7B01022F047022FD1E
:1015700005C080910B0190910C0102C080E090E0C9
:101580002A8349830E94220A2A814981811138C015
:101590001092AF034093B103F092B303E092B20311
:1015A000812F880F81608093B4039091B00321FF55
:1015B00002C085E001C084E0892B8093B003809154
:1015C000B00381FF0BC08091B0038D7F8093B00387
:1015D0008091B4038093BB0085EC01C085EE8093BD
:1015E000BC00822F817020FF0BC0011105C08091CB
:1015F0000B0190910C0102C080E090E00E94220A51
:101600002296E6E00C945721A0E0B0E0EAE0FBE08F
:101610000C9439210E94761B0091AB031091AC030E
:101620002091AD033091AE036B017C01C01AD10A49
:10163000E20AF30A9701860141E1C41647E2D406A3
:10164000E104F10408F442C02091AA0331E0320F12
:101650003093AA0320FF02C017E001C010E060939E
:10166000AB037093AC038093AD039093AE0363E040
:1016700070E082E194E00E94020161E070E082E1AA
:1016800094E00E94020107E0010F812F90E0EC013D
:10169000CC0FDD1FC35FDE4F68817981672F77270D
:1016A00063707727880F991F880F991F682B792BF4
:1016B00082E194E00E94FA0068817981772782E1D3
:1016C00094E00E94FA001F5F1013DFCFCDB7DEB7A2
:1016D000E8E00C94552125B190E0FC01EE0FFF1FCE
:1016E000E80FF91FE65EFC4F8081282B25B988B1F1
:1016F0009181892B88B98BB19281892B8BB90895FF
:1017000085B190911703892385B988B19091180309
:10171000892388B98BB19091190389238BB90895D6
:101720001F920F920FB60F9211242F933F934F9356
:101730005F936F937F938F939F93AF93BF93CF9359
:10174000EF93FF93C091760380910601C81708F0CC
:101750003EC080911503909116039093870080936B
:101760008600EC2FF0E0EE0FFF1FE35FFE4F80815D
:1017700091810E94DF02880F991F90931603809336
:101780001503809115039091160320910701309164
:101790000801281B390B3093080120930701809121
:1017A000000490910104880F991F2817390720F42D
:1017B000909308018093070180917403811142C0C6
:1017C0008091F80380FF41C0C830E0F53EC08091B1
:1017D0001503909116039093870080938600809163
:1017E000070190910801909316038093150380914F
:1017F0007403882319F08FEF9FEF06C080911503C3
:1018000090911603885592409093890080938800A8
:1018100080E49CE990930801809307018091840003
:10182000909185008097D0F30E94800B8091750382
:10183000811105C08091060181500E946B0B1092AE
:10184000760327C08FEF9FEF06C08091150390911C
:101850001603885592409093890080938800809168
:101860008400909185008097D0F30E94800B809136
:101870007503811104C080917603811106C08091A7
:1018800076038F5F8093760304C081500E946B0BB8
:10189000F6CFFF91EF91CF91BF91AF919F918F9133
:1018A0007F916F915F914F913F912F910F900FBE5C
:1018B0000F901F90189524E0829FC00111248C3056
:1018C000910538F0853F23E0920728F084EF93E0FC
:1018D00008958CE090E00895CF93DF93C091F903D1
:1018E000C03390F48C2F807339F0803141F48091B3
:1018F00077038295807F05C080917C0302C0809130
:101900007D03CF70D0E015C0CF33E0F4CF70D0E0CE
:10191000809177038295807F0E945B0CDE01AA0F85
:10192000BB1FA35FBE4F11969C938E93219680910F
:101930007D030E945B0CFE01EE0FFF1FE35FFE4F75
:1019400091838083DF91CF91089580917803909166
:1019500079039F770E940003809377038F3029F4E7
:1019600080917D038695805804C099E0899F802DE1
:10197000112480937C03F8940E946C0C78948091DD
:10198000ED038132E1F480917C039FEF980F9E3F3D
:1019900078F08091B0008F7D8093B00061E08091FD
:1019A0007C03811101C060E083E00E94671C089500
:1019B0008093B4008091B00080628093B00008955D
:1019C000FF920F931F93CF93DF930BEE13E0C0E0D2
:1019D000D0E0B3E0FB2E8C2FD801ED918D019E2F2E
:1019E000907F9031F1F4EF70F0E0EE0FFF1FE35FB6
:1019F000FE4F208131816F2D0E94CE20E92FF0E033
:101A0000EE0FFF1FEC56FD4F61E080819181821740
:101A1000930708F060E0FE01EE55FD4F80810E94C3
:101A2000671C2196C830D105B1F6CDB7DEB7E5E029
:101A30000C9458210F931F93CF93DF9303E513E08A
:101A4000C0E0D0E02091F903822F8F7090E0C8179A
:101A5000D907E9F00196C817D90711F42033B8F473
:101A6000F801808191819F70892B79F0F894F801B9
:101A7000808191819F700E94B402FE01EE0FFF1FD2
:101A8000E35FFE4F9183808378940E94E00C21965F
:101A90000E5F1F4FC031D105A9F6DF91CF911F9185
:101AA0000F910895FF920F931F93CF93DF9381ECD3
:101AB00093E00E94AC01809306019091F903292FD5
:101AC0002F70281304C081E0820F80930601905389
:101AD0009F3060F44091060130E0842F90E0019740
:101AE0002817390719F44F5F4093060180910601CA
:101AF000813118F080E180930601ECE1F3E0DF0131
:101B000012971C92DF0111971C921082339683E08A
:101B1000E433F807A1F74FEF3FEFACEAB2E00BEE8A
:101B200013E02FEFE80189918E018031F8F490E005
:101B3000FD0132976081FC01EE0FFF1FE80FF91FD6
:101B4000E65EFC4F8081862B8083CD010197EC01FE
:101B500058818181852B81839C918281892B82830D
:101B60006095509590952923352346231396D3E00D
:101B7000033F1D07B9F640931703309318032093D2
:101B80001903C2EAD2E00BEE13E0F12CF8018191C7
:101B90008F01823230F08632B8F0863211F460E084
:101BA00010C0F6E0FF1204C08091C1008F7E06C015
:101BB00087E0F81205C08091C100877F8093C10043
:101BC00061E088810E942E1CF3942196E8E0FE12C9
:101BD000DDCF8091EB03803231F461E089E00E9437
:101BE000671C82E801C082E08093800081E08093DE
:101BF0007503809374038091ED03813211F0873275
:101C0000D9F461E083E00E942E1C60E083E00E9432
:101C1000671C8091ED03813231F481E08093B00044
:101C20008093B10009C082E08093B00085E080938A
:101C3000B1008EE38093B3008AE1809381008FEF3F
:101C40009FEF909389008093880080ED97E09093B8
:101C500087008093860080E49CE99093080180933C
:101C600007019093160380931503109276038091D9
:101C70006F00816080936F008091F80383FF0DC037
:101C800080915303909154039F70892B31F00E94EF
:101C90001A0D1092740310927503CDB7DEB7E5E00C
:101CA0000C945821CF93C82F8091F0038B3221F4EC
:101CB0006C2F8FE00E94671C8091ED03873249F4FE
:101CC0008091B000CC2311F0806101C08F7E8093A1
:101CD000B000CF910895A4E2B0E0E1E7FEE00C94FB
:101CE0002F216B017C010E946A1B4B015C0181E08A
:101CF0000E94660483E08093BE030E9464056AEC40
:101D000071E082E194E00E94381D7BE1272EE0E53E
:101D10003E2EF7E47F2EA6E44A2EB5E55B2EC114D5
:101D2000D104E104F10469F00E946A1B6819790981
:101D30008A099B096C157D058E059F0510F080E0D2
:101D4000D5C08091BE03843051F768ED71E082E127
:101D500094E00E94381D8FE70E944D030E946003AB
:101D60008CA3823601F501EC13E00E946003D801D8
:101D70008D938D01B3E00A3E1B07B9F78091C10333
:101D8000883309F0ADC061EE71E082E194E00E9419
:101D9000381D82E48CA361E0CE0184960E94C305C5
:101DA0005D9A81E0A3C0803741F0893611F581E06A
:101DB0000E947B0889E4898304C03982C12CD12C1C
:101DC00076019091BD038091F803992311F080680A
:101DD00001C08F778093F803EAEEF3E0DE011296FC
:101DE000822D01900D928A95E1F76CE1CE0101966A
:101DF00075C08437E1F4E4E5E98383E08A8388E809
:101E00008B8388E08C838FE08D838EE1EDE2F1E0BF
:101E1000DE01169601900D928A95E1F763E2CE01FC
:101E200001960E94C305C12CD12C760159C085377B
:101E300089F40AEE13E00E946003D8018D938D01AE
:101E4000B4E005301B07B9F761E080E00E94CD07E0
:101E50005CA241C08636B9F44982E3E5F3E0AE0105
:101E60004D5F5F4F208131813296CA010197DC01BD
:101E70003C93DA012C934E5F5F4FB3E0E337FB07EF
:101E800089F761E2B3CF8736C9F403E513E00E9416
:101E90006003682E0E946003262D30E0322F222737
:101EA000280F311DF801219331938F01F3E003379F
:101EB0001F0769F77CA20E9467080DC0873481F470
:101EC000E3E5F3E01192119283E0E337F807D1F7ED
:101ED0000E9467087CA261E0CE0184960E94C3053F
:101EE00083E08093BE030E94410519CFA496E2E1EE
:101EF0000C944B211F93CF93DF93C82FD62F61E013
:101F00000E942E1C61E08C2F0E94671C61E08D2FC7
:101F10000E94671C8AE090E00E94BF1B8D2F0E94E8
:101F20009A1C892B71F060E08C2F0E94671C8AE05C
:101F300090E00E94BF1B8D2F0E949A1C11E0892BFC
:101F400009F010E060E08C2F0E942E1C60E08C2FC6
:101F50000E94671C60E08D2F0E94671C812FDF911B
:101F6000CF911F91089580E48093BA001092BD0034
:101F70008DE990E09093B6038093B50310925003DF
:101F800015E004E0C2E0FC2E80915003813039F46A
:101F900080E00E946604F09250035E98F5CFC091F5
:101FA0005003C33061F45D98809192030E948803CE
:101FB000C093BE030E94410500935003E5CF80917A
:101FC0005003843009F78091BE038430E9F68FE72F
:101FD0000E944D03C0E0D3E0E091E903E770F0E038
:101FE000E656FD4F808190E09E0120503340281737
:101FF000390724F40E9460038993EECF10935003B5
:102000005D9AC2CFAAE2B0E0E8E0F0E10C943E2194
:102010001FEF198389E2E1ECF3E0DE0112960190F3
:102020000D928A95E1F721E04AE2BE016F5F7F4F92
:1020300080E20E94580A81110EC021E041E0BE01F9
:102040006F5F7F4F80E20E94AD0A811104C082E081
:102050008093500302C0109350038091500382304C
:1020600051F00E946A1B60934C0370934D03809360
:102070004E0390934F03AA96E3E00C945A21A1E0FB
:10208000B0E0E5E4F0E10C943F2180915003823010
:10209000D9F480919203805A898321E041E0BE0106
:1020A0006F5F7F4F80E20E94580A882369F08FEFAC
:1020B000809350030E946A1B60934C0370934D03FE
:1020C00080934E0390934F032196E2E00C945B21A2
:1020D000A1E0B0E0EEE6F0E10C943F2180915003E6
:1020E0008230D1F421E041E0BE016F5F7F4F80E29A
:1020F0000E94AD0A882371F08FEF809350030E94F5
:102100006A1B60934C0370934D0380934E0390932E
:102110004F0302C0898101C08FEF2196E2E00C9449
:102120005B21A2E2B0E0E7E9F0E10C942F219E01EF
:102130002F5F3F4F80E1D9011D928A95E9F76CEE40
:1021400071E082E194E029A33AA30E94381D0E9425
:1021500064051D8A1E8A1F8A188E312C212C00E0EE
:10216000812C912C540180E4482E81EE582E8DE96B
:10217000682E88E1782E90E5C92E93ECD92EE12CBB
:10218000F12C84EF91E0A0E0B0E08D8F9E8FAF8FB7
:10219000B8A380EC91EDA8E9BBE1898F9A8FAB8F52
:1021A000BC8F80E491EEADE9B8E1898B9A8BAB8B63
:1021B000BC8B82E194E00E94041E892B09F4E1C0EB
:1021C00082E194E00E94311E9C0133272C323105BC
:1021D00009F442C0ACF42332310509F0ABC01982D6
:1021E0001A821B821C821D821E821F8218861986FB
:1021F0001A861B861C861D861E861F86188A60C04E
:102200002434310529F02335310509F4B2C092C0D8
:1022100064E482E194E00E941C1D2AE030E040E486
:1022200051EE6DE978E182E194E00E94981D6CE244
:1022300082E194E00E941C1D2AE030E040EC51ED68
:1022400068E97BE182E194E00E94981D6CE282E102
:1022500094E00E944A1DADCF0F5F043009F0A9CF72
:1022600029813A814B815C81A8EEB3E00E94AB20CA
:10227000698B7A8B8B8B9C8B2D813E814F8158850E
:102280000E94AB20698F7A8F8B8F9C8F29853A852E
:102290004B855C852D8F3E8F4F8F58A32D853E85B6
:1022A0004F8558890E94AB206B017C0160323EE46F
:1022B00073078105910530F462E38CE10E94750398
:1022C00000E077CF603345E774078105910510F48E
:1022D00062E2F3CF60345CE975078105910510F483
:1022E00066E2EBCF80E5C81683ECD806E104F10482
:1022F00010F462E1E2CF90E6C9169AEED906E10445
:10230000F10410F465E1D9CFA0E7CA16A1E1DA061D
:10231000A1E0EA06F10410F461E0CFCFB0EACB16F9
:10232000B6E8DB06B1E0EB06F10410F463E0C5CFDC
:1023300065E0C3CF10ED180F1A3008F03ACFE1E096
:10234000F0E0EC0FFD1F24E0029FE00DF11D1124D1
:102350002081318142815381AAE0B0E00E94AB200C
:10236000610F711D811D911D608371838283938331
:1023700020CF49885A886B887C88812C912C540105
:1023800018CF81149104A104B10489F4C301B201EE
:102390000E94FB0361E070E080E090E00E94991BE6
:1023A0001D8A1E8A1F8A188E312C22242A948D8D14
:1023B0009E8DAF8DB8A188169906AA06BB06D0F4EB
:1023C0000E949E032D893E894F89588D280F311D0B
:1023D000411D511D2D8B3E8B4F8B588F381608F4A5
:1023E000382E821508F4282E3FEF831A930AA30A89
:1023F000B30A56C0C301B20128EE33E040E050E01A
:102400000E94EE20BA01A9012AE030E082E194E0C6
:102410000E94E61D6CE282E194E00E941C1D4AE0ED
:1024200050E0632D82E194E00E94F51D6CE282E1B0
:1024300094E00E941C1D6D897E898F89988DA5016D
:1024400094010E94EE20BA01A9012AE030E082E165
:1024500094E00E94E61D6CE282E194E00E941C1D63
:102460004AE050E0622D82E194E00E94F51D6CE2AA
:1024700082E194E00E944A1D4C0C5D1C6E1C7F1C86
:10248000898D9A8DAB8DBC8D84159505A605B705F4
:1024900020F449885A886B887C88812C912C5401BF
:1024A00029893A894B895C89283E33404105510589
:1024B00009F07FCEA296E2E10C944B21A1E0B0E0BE
:1024C000E4E6F2E10C943F2180E00E94920161E099
:1024D00085E00E942E1C61E086E00E942E1C0E9476
:1024E000690160E080E00E942E1C61E081E00E94B2
:1024F0002E1C40E052EC61E070E082E194E00E942A
:102500004C1F0E94B9080E946C0869EF71E082E1DB
:1025100094E00E94191D88E893E00E94680760E13A
:1025200072E082E194E00E94191D4AE050E065E00B
:1025300070E082E194E00E94CE1D0E947E017894BA
:102540005E9A63E183E00E947A0F882329F05E9807
:102550005D980E949110FBCF62E189E00E947A0FA2
:10256000811104C00E945508811119C063E572E011
:1025700082E194E00E94191D60E070E0CB010E94AE
:102580006B0E882349F00E94620868E172E082E1E4
:1025900094E00E94381D5D9A0E94520D10C00E9466
:1025A000520D8091EC03823209F0C6C08091EE0397
:1025B000833209F0C1C08091F80381FDC3C08091CE
:1025C000EC03823231F58091EE03833211F581E024
:1025D0000E94C3088091F80382FF08C063E372E0A1
:1025E00082E194E00E94381D0E94B30F64E170E024
:1025F00080E090E00E94991B21E041E0BE016F5F06
:102600007F4F80E20E94AD0A811103C081E0809378
:1026100050036EE372E082E194E00E94191D8FE0A6
:102620000E94920180E00E9466041092920380E072
:102630000E94880380E0883170F08093D40283E0A8
:102640008093BE030E94640580915003882371F03B
:102650000E9402100BC021E0280FE82FF0E0EF539A
:10266000FC4F9785992349F3822FE5CF8091F203A0
:10267000982F9D7F983229F440E052EC61E070E0A1
:1026800023C0893251F42EE240EA56E861E070E05E
:1026900082E194E00E94CD1F1BC08091E903887104
:1026A000803129F440E855E260E070E00DC04091CF
:1026B000C2035091C3036091C4037091C5034A30B3
:1026C00051056105710570F382E194E00E944C1F91
:1026D00082E194E00E94041E892B29F082E194E0BB
:1026E0000E94311EF5CF8091F103843229F0809150
:1026F000C1008F7E8093C1008091F203853241F04A
:102700008852833028F08091C100877F8093C10078
:102710001092D6021092D502109252030E94761B9C
:1027200060938E0370938F03809390039093910333
:102730002196E2E00C945B218091F8038B7F8093DB
:10274000F80339CF82FD3BCF64EF71E080E090E089
:102750000E946B0E882309F432CF0E94620868E160
:1027600072E082E194E00E94381D0E94520D5D9A51
:1027700026CFCF93DF9382E194E00E94041E892B41
:10278000E9F0C091D502D0E0CE0101968F71992772
:102790002091D60230E08217930781F082E194E025
:1027A0000E94311EC952DD4F88838091D50290E08E
:1027B00001968F7199278093D502DDCFDF91CF915C
:1027C0000895A0E0B0E0E7EEF3E10C943921D82FB2
:1027D000C62F0E94761B0091AB031091AC03209191
:1027E000AD033091AE036B017C01C01AD10AE20A3D
:1027F000F30A9701860141E1C41647E2D406E104D9
:10280000F10408F4D1C16093AB037093AC038093DF
:10281000AD039093AE0380910D0190910E01880F4E
:10282000991F80939303892F877020919403287FA9
:10283000282B2093940380910F0190911001880F11
:10284000991F382F330F330F330F2770232B20930B
:102850009403282F22952695277080919503807CDC
:102860009770990F990F990F822B892B809395035D
:102870002091110130911201220F331F922F929556
:10288000990F990F907C8F73892B80939503932FC9
:102890009295990F990F907C822F86958695892B1A
:1028A0008093960332FB882780F9209197032E7F2F
:1028B000282B209397038091130190911401880F86
:1028C000991F382F330F2170232B20939703382F14
:1028D000331F3327331F20919803207F892F877060
:1028E000880F232B282B209398038091150190911A
:1028F0001601880F991F382F3295307F2F70232BA8
:1029000020939803382F32953F70209199032078B7
:10291000892F87708295807F232B282B2093990302
:102920008091170190911801880F991F2F7720939C
:102930009903292F2795222727958695822B809307
:102940009A03892F8695837020919B032C7F282BD7
:1029500020939B038091190190911A01880F991F70
:10296000382F330F330F2370232B20939B03382FE3
:10297000329536953695337020919C03207E892FB1
:102980008770880F880F232B282B20939C0380911E
:102990001B0190911C01880F991F382F3295330F1E
:1029A000307E2F71232B20939C039295990F907E5C
:1029B000869586958695892B80939D0380911D0130
:1029C00090911E01880F991F80939E03892F877015
:1029D00020919F03287F282B20939F0380911F0124
:1029E00090912001880F991F382F330F330F330F29
:1029F0002770232B20939F03282F2295269527703D
:102A00008091A003807C9770990F990F990F822B6A
:102A1000892B8093A0032091210130912201220F64
:102A2000331F922F9295990F990F907C8F73892B5A
:102A30008093A003932F9295990F990F907C822FEA
:102A400086958695892B8093A10332FB882780F990
:102A50002091A2032E7F282B2093A2038091230193
:102A600090912401880F991F382F330F2170232B49
:102A70002093A203382F331F3327331F2091A30342
:102A8000207F892F8770880F232B282B2093A30367
:102A90008091250190912601880F991F382F32953A
:102AA000307F2F70232B2093A303382F32953F7054
:102AB0002091A4032078892F87708295807F232B13
:102AC000282B2093A4038091270190912801880F3F
:102AD000991F2F772093A403292F27952227279525
:102AE0008695822B8093A503969593708091A6037B
:102AF0008C7F892B8093A6032091290130912A0194
:102B0000220F331F922F990F990F8370892B809377
:102B1000A60322952695269523708091A703807E93
:102B2000932F9770990F990F822B892B8093A7036E
:102B300020912B0130912C01220F331F922F92955F
:102B4000990F907E8F71892B8093A703832F829595
:102B5000880F807E269526952695282B2093A803FE
:102B6000DD2311F088E001C080E0CC2311F094E077
:102B700001C090E0892B8093A9036FE070E082E1AF
:102B800094E00E940201C3E9D3E0699182E194E0FC
:102B90000E945E1E83E0CA3AD807B9F760E070E091
:102BA00082E194E00E940201CDB7DEB7E8E00C9428
:102BB0005521CF93C82F682F82E194E00E945E1EBA
:102BC0008C2F0E940A01CF910895A0E0B0E0EBEEB7
:102BD000F5E10C943921C82F0E94761B0091AB03BC
:102BE0001091AC032091AD033091AE036B017C01D9
:102BF000C01AD10AE20AF30A9701860141E1C4161C
:102C000047E2D406E104F10408F445C06093AB0345
:102C10007093AC038093AD039093AE031092C00306
:102C20001092BF0388EA0E94D915CC2311F081E8E5
:102C300001C081E00E94D91580E10E94D91500E011
:102C400010E0F801EE0FFF1FE35FFE4F80819181DE
:102C50000E94DF02EC01B3E0CC0FDD1FBA95E1F773
:102C60008D2F0E94D9158C2F0E94D9150F5F1F4FF1
:102C70000031110531F76091C00370E082E194E00A
:102C80000E94FA006091BF037091C003772782E130
:102C900094E00E94FA00CDB7DEB7E8E00C9455212D
:102CA000AAE1B0E0E6E5F6E10C9431210E949B0038
:102CB0008CE00E946F0381110BC06CE872E082E12E
:102CC00094E00E94381D80E00E9466040E94640522
:102CD0000E94B9130E94761B0E94681091E0853013
:102CE00009F090E01FEF8091BE03843009F4FEC12B
:102CF0009111FCC17CC00E94A20390937B0380933E
:102D00007A035D9AC0928E03D0928F03E092900373
:102D1000F09291031092510380917803909179037E
:102D2000880F991F816090937903809378035E9850
:102D300080E00E94520E80910003982F9E7309F04C
:102D40002CC2F8948091E90341E053E06DE071E01A
:102D500087700E942E020E946C0C78949091000360
:102D600080914A0390FF13C2811124C093E5E92E9C
:102D700093E0F92E00E010E0F7018081918194FD4D
:102D80000CC0F801EE0FFF1FE35FFE4F80819181C1
:102D90000E94DF02D7018D939C930F5F1F4FB2E01B
:102DA000EB0EF11C0031110539F70E94670881E034
:102DB00080934A0380915203811103C081E0809384
:102DC0005203109273031092750310927403809152
:102DD000E903887109F009C20E94E00C83E0809346
:102DE000BE030E94410581E080934B035D980E94E1
:102DF000761B4B015C010E946A1B6B017C01809178
:102E00005103823008F063C040908E0350908F03CE
:102E1000609090037090910380918A0390918B034E
:102E2000A0918C03B0918D0384159505A605B70577
:102E300009F44DC081EC93E00E94BC016C5D7540CB
:102E40008109910995018401041915092609370999
:102E50006017710782079307D0F540928A0350925A
:102E60008B0360928C0370928D030E949E03282F27
:102E700080937E0380917F0390918003820F911D48
:102E80009093800380937F03609181036F5F6093D1
:102E900081036930E0F070E00E94DA2070938003D3
:102EA00060937F0380917D03E3E08E9F600D711D31
:102EB0001124769567957695679560937D030E94BA
:102EC000A50C1092800310927F03109281038091D1
:102ED00052030091D402882351F11091510310172D
:102EE00008F035C240908E0350908F03609090039D
:102EF00070909103A50194012419350946095709D9
:102F00002F8B388F498F5A8F81EC93E00E94BC0140
:102F100068517C4F8F4F9F4F2F89388D498D5A8D27
:102F2000621773078407950708F4D8C110C280910F
:102F30008E0390918F03A0919003B091910375013E
:102F40006401C81AD90AEA0AFB0A81EC93E00E94DC
:102F5000BC019B01AC01A02FB0E00E94AB206C151E
:102F60007D058E059F0558F480928E0390928F0305
:102F7000A0929003B092910381E080934B038091E3
:102F80007403811116C08091F203883219F40E94F3
:102F9000040B0FC0893239F460915103809173039F
:102FA0000E94E11306C08A3221F4809173030E94CB
:102FB000E51580914B03882309F472C0E0919203D8
:102FC000EF5FE0939203E83131F0F0E0EF53FC4F14
:102FD0008785811102C0109292038091FA0390912B
:102FE000FB03A091FC03B091FD03892B8A2B8B2B53
:102FF00009F44EC08091820390918303A0918403D1
:10300000B0918503892B8A2B8B2B09F441C00E9438
:103010005406082F10E02091090130910A013695DD
:103020002795369527952C5E3F4F2017310770F472
:103030000E946A1B68517C4F8F4F9F4F60938203A1
:10304000709383038093840390938503C801880F52
:10305000991F880F991F4091090150910A019A0107
:10306000220F331F240F351F820F931F96958795CC
:103070009695879590930A01809309016091C60304
:103080007091C7038091C8039091C9030E94FB030C
:10309000809192030E9488030E943F1010924B037C
:1030A000809150038F3F09F04DC20E946A1B00912E
:1030B0004C0310914D0320914E0330914F03601B40
:1030C000710B820B930B693E73408105910508F4E7
:1030D00039C20E946A1B60934C0370934D03809326
:1030E0004E0390934F030E9402102CC20E94761B45
:1030F0006B017C018091BE038430D1F48FE70E9484
:103100004D0300E013E0E091E903E770F0E0E656DC
:10311000FD4F808190E098012050334028173907F7
:103120000CF0E9CD0E946003D8018D938D01EBCFA7
:10313000E091E903E770F0E0E656FD4F40814F5F14
:1031400021E0BE016F5F7F4F80E20E94AD0A8823BD
:1031500071F0109350030E946A1B60934C037093AC
:103160004D0380934E0390934F0390E0BCCDE091CC
:10317000E903E770F0E0E656FD4F408150E0BE0104
:103180006E5F7F4F80E093E00E946C21BBCD88236F
:1031900009F410CE10924A030DCE982F98739833ED
:1031A00009F008CE9091F702892787FF03CE905847
:1031B0009093F7028091F203853209F0FBCD10E085
:1031C000212F30E080910003877090E082179307F1
:1031D0000CF4F0CD1F5FE12FF0E0E050FD4F608177
:1031E00082E194E00E945E1EEBCF8091F702909105
:1031F0000003982796FD66C0807C90E48927809321
:10320000F7028091D6023091D5028317D1F0E8EF12
:10321000F2E020E02F5F90E0DC01A952BD4F4C911D
:10322000419301968F719927283011F08313F2CFC3
:103230008093D602295C8091F702282B2093F70215
:1032400041C080917E038093F8028091EC03863226
:1032500011F482E105C08091EF03863251F48EE0D3
:103260000E94C31C95958795959587958093F90243
:1032700002C01092F9028091EE03863211F483E1CC
:1032800005C08091F003863251F48FE00E94C31C88
:1032900095958795959587958093FA0202C010922F
:1032A000FA0280917A0390917B039093FB028093C2
:1032B000FC0280917803909179039F770E9400032C
:1032C0008093FD0269E087EF92E00E947C050E94F6
:1032D000EB05811181CD0E94B913F9CF809178035C
:1032E00090917903880F991F9093790380937803C5
:1032F00081E080934B03111110C0C0928603D092DD
:103300008703E0928803F09289031092820310925F
:10331000830310928403109285031F5F109351035F
:1033200081EC93E00E94BC01640D751D861D971D04
:1033300060938E0370938F03809390039093910317
:103340005E9A81E00E94520E0E94A50C03C01017E5
:1033500009F4A7C080915103882309F410CE80910D
:1033600002048823D9F090917303911117C0409102
:103370008603509187036091880370918903460109
:103380005701841A950AA60AB70A90E00E94230101
:10339000681579058A059B0508F4B5C08091040479
:1033A0008823D9F090917503911117C0409186033D
:1033B00050918703609188037091890346015701FA
:1033C000841A950AA60AB70A90E00E94230168159C
:1033D00079058A059B0508F4ADC080910304882314
:1033E000D9F090917403911117C0409186035091C8
:1033F0008703609188037091890346015701841AFD
:10340000950AA60AB70A90E00E942301681579057B
:103410008A059B0508F492C08091FA039091FB0302
:10342000A091FC03B091FD03892B8A2B8B2B09F40F
:10343000A6CD8091820390918303A0918403B091E3
:1034400085030097A105B10509F499CDC81AD90AD9
:10345000EA0AFB0AF7FC93CD8091F803829581700C
:103460000E94970680E00E9466040E9441050E9427
:103470006A1B6B017C012091FF0330E0A8EEB3E0F2
:103480000E949C20C60ED71EE81EF91E6894C0F844
:10349000C0928203D0928303E0928403F09285036A
:1034A0006ECD80918E0390918F03A0919003B09187
:1034B000910324013501481A590A6A0A7B0A81ECF2
:1034C00093E00E94BC019B01AC01A12FB0E00E94DF
:1034D000AB20641575058605970508F03BCF109263
:1034E00079031092780381E080934B0310927D035F
:1034F0000E94A50C80928E0390928F03A09290035D
:10350000B092910327CF81E0809373030E941A0D3C
:103510008091FE030E9448016C0D7D1D8E1D9F1D34
:10352000616060938203709383038093840390931C
:10353000850334CF81E0809375034FCF81E0809382
:1035400074036ACF6A96E0E10C944D218230E8F46E
:10355000E82FF0E0EE0FFF1FEB5FFB4F71836083FE
:10356000813041F0809169008C7F842B80936900C9
:10357000E89A089580916900440F551F440F551F24
:10358000837F842B80936900E99A08951F920F929C
:103590000FB60F9211242F933F934F935F936F9326
:1035A0007F938F939F93AF93BF93EF93FF938091FC
:1035B000050490910604892B29F0E0910504F0910F
:1035C00006040995FF91EF91BF91AF919F918F9163
:1035D0007F916F915F914F913F912F910F900FBE0F
:1035E0000F901F9018951F920F920FB60F921124F3
:1035F0002F933F934F935F936F937F938F939F93FB
:10360000AF93BF93EF93FF938091070490910804C9
:10361000892B29F0E0910704F09108040995FF91A6
:10362000EF91BF91AF919F918F917F916F915F913A
:103630004F913F912F910F900FBE0F901F901895B3
:103640001F920F920FB60F9211242F933F938F93D7
:103650009F93AF93BF9380910A0490910B04A09124
:103660000C04B0910D043091090423E0230F2D3791
:1036700020F40196A11DB11D05C026E8230F029676
:10368000A11DB11D2093090480930A0490930B049B
:10369000A0930C04B0930D0480910E0490910F043C
:1036A000A0911004B09111040196A11DB11D809349
:1036B0000E0490930F04A0931004B0931104BF91D3
:1036C000AF919F918F913F912F910F900FBE0F90CF
:1036D0001F9018952FB7F89460910A0470910B040D
:1036E00080910C0490910D042FBF08953FB7F8947A
:1036F00080910E0490910F04A0911004B0911104D8
:1037000026B5A89B05C02F3F19F00196A11DB11D3C
:103710003FBF6627782F892F9A2F620F711D811D59
:10372000911D42E0660F771F881F991F4A95D1F7B8
:103730000895CF92DF92EF92FF92CF93DF936B01C8
:103740007C010E94761BEB01C114D104E104F10459
:1037500079F00E94761B6C1B7D0B683E7340A0F3D2
:1037600081E0C81AD108E108F108C851DC4FECCF5C
:10377000DF91CF91FF90EF90DF90CF900895019768
:10378000009739F0880F991F880F991F02970197AA
:10379000F1F70895789484B5826084BD84B5816022
:1037A00084BD85B5826085BD85B5816085BDEEE649
:1037B000F0E0808181608083E1E8F0E01082808128
:1037C00082608083808181608083E0E8F0E0808196
:1037D00081608083E1EBF0E0808184608083E0EBB6
:1037E000F0E0808181608083EAE7F0E0808184609E
:1037F00080838081826080838081816080838081FA
:10380000806880831092C1000895833081F028F48D
:10381000813099F08230A1F008958630A9F0873088
:10382000B9F08430D1F4809180008F7D03C0809105
:1038300080008F7780938000089584B58F7702C0D1
:1038400084B58F7D84BD08958091B0008F7703C0CB
:103850008091B0008F7D8093B0000895CF93DF9367
:1038600090E0FC01E458FF4F2491FC01E057FF4F2A
:103870008491882349F190E0880F991FFC01E85456
:10388000FF4FA591B49182559F4FFC01C591D491F2
:103890009FB7611108C0F8948C91209582238C9376
:1038A000888182230AC0623051F4F8948C91322FBF
:1038B000309583238C938881822B888304C0F8946D
:1038C0008C91822B8C939FBFDF91CF910895A1E0C3
:1038D000B0E0EDE6FCE10C943D21282F30E0F90149
:1038E000E859FF4F8491F901E458FF4F1491F90111
:1038F000E057FF4F04910023C9F0882321F069832A
:103900000E94051C6981E02FF0E0EE0FFF1FE255D9
:10391000FF4FA591B4919FB7F8948C91611103C0AA
:103920001095812301C0812B8C939FBF2196E4E0E9
:103930000C945921CF93DF93282F30E0F901E859F7
:10394000FF4F8491F901E458FF4FD491F901E057FA
:10395000FF4FC491CC2391F081110E94051CEC2FE4
:10396000F0E0EE0FFF1FEC55FF4FA591B4912C91A5
:103970002D2381E090E021F480E002C080E090E01F
:10398000DF91CF9108958E3008F08E50877020918E
:10399000BD0190E4299F90011124822B80937C002B
:1039A00080917A00806480937A0080917A0086FD0D
:1039B000FCCF809178002091790090E0922B0895BF
:1039C000A0E0B0E0E6EEFCE10C9439216C017A0154
:1039D000EB01E60EF71E00E010E0CE15DF0561F00A
:1039E0006991D601ED91FC910190F081E02DC60125
:1039F0000995080F191FF1CFC801CDB7DEB7E8E070
:103A00000C9455216115710589F0DB010D900020A2
:103A1000E9F7AD0141505109461B570BDC01ED910F
:103A2000FC910280F381E02D0995089580E090E0FB
:103A300008950E94021D0895DC01ED91FC91019012
:103A4000F081E02D099508950F931F93CF93DF9395
:103A5000EC016DE00E941C1D8C016AE0CE010E9409
:103A60001C1D800F911FDF91CF911F910F91089521
:103A70000F931F93CF93DF93EC010E94021D8C01E3
:103A8000CE010E94241D800F911FDF91CF911F91C5
:103A90000F9108950F931F93CF93DF93EC010E9432
:103AA0001C1D8C01CE010E94241D800F911FDF91EF
:103AB000CF911F910F910895A1E2B0E0E2E6FDE100
:103AC0000C9435217C01C42EE52FCB01D22E19A2F6
:103AD00021E02D1510F02AE0D22E8E010F5D1F4F30
:103AE0008D2C912CA12CB12C6C2D7E2FA501940135
:103AF0000E94EE208C2DD29E8019112401501109B4
:103B00008A3010F4805D01C0895CF8018083211542
:103B100031054105510521F0C22EE32FCA01E4CF42
:103B2000B801C7010E94021DA196ECE00C9451213E
:103B3000A0E0B0E0EEE9FDE10C943921EC016A016E
:103B40007B012115310541F4E881F9810190F08173
:103B5000E02D642F09951DC02A303105A9F477FFA7
:103B600012C06DE20E941C1D8C0144275527BA012A
:103B70004C195D096E097F092AE0CE010E945C1D87
:103B8000800F911F06C02AE0B701A601CE010E9456
:103B90005C1DCDB7DEB7E8E00C9455210F931F9361
:103BA000CF93DF93EC019A01AB01662757FD609537
:103BB000762F0E94981D8C01CE010E94241D800F3B
:103BC000911FDF91CF911F910F910895211531051C
:103BD00049F4DC01ED91FC910190F081E02D642F1E
:103BE000099508950E945C1D08959A01462F50E0A2
:103BF00060E070E00E94E61D08959A01AB0160E06C
:103C000070E00E94E61D0895FC0124853585F901C8
:103C1000E05CFF4F80819181F901EE5BFF4F2081D5
:103C20003181821B930B8F7399270895FC01848542
:103C30009585FC01E05CFF4F40815181FC01EE5B0A
:103C4000FF4F208131814217530741F00190F081ED
:103C5000E02DE80FF91F808190E008958FEF9FEF2E
:103C60000895FC0184859585FC01E05CFF4F40814F
:103C70005181FC01EE5BFF4F2081318142175307D8
:103C800079F0A081B181A80FB91F8C912081318179
:103C90002F5F3F4F2F7333273183208390E00895A8
:103CA0008FEF9FEF0895FC0181A1882329F0A4895B
:103CB000B5898C9186FFFBCF11A20895CF93DF9336
:103CC000FC0126853785D901A05CBF4F8D919C9161
:103CD000119701968F739927E901CE5BDF4F4881D9
:103CE000598184179507D9F30D90BC91A02DA20F8F
:103CF000B31F6C93A685B785A05CBF4F11969C93AC
:103D00008E93A689B7892C9181E090E0078C02C040
:103D1000880F991F0A94E2F7282B2C9381E081A346
:103D20000488F589E02D80818064808381E090E0C3
:103D3000DF91CF91089508951F920F920FB60F92C1
:103D400011242F933F934F938F939F93EF93FF9360
:103D50008091C00082FD1CC04091C6008091B804D3
:103D60009091B90401968F7399272091BA043091EC
:103D7000BB048217930771F0E091B804F091B90485
:103D8000E858FB4F40839093B9048093B80402C075
:103D90008091C600FF91EF919F918F914F913F913C
:103DA0002F910F900FBE0F901F90189582E194E015
:103DB0000E94041E892B11F00E949B1E08951F92E1
:103DC0000F920FB60F9211242F933F938F939F93CF
:103DD000EF93FF93209174043091750480917604E1
:103DE000909177042817390731F48091C1008F7DB5
:103DF0008093C10014C0E0917604F0917704EC5CEC
:103E0000FB4F2081809176049091770401968F7307
:103E1000992790937704809376042093C600FF91AE
:103E2000EF919F918F913F912F910F900FBE0F9027
:103E30001F901895A0E0B0E0E0E2FFE10C9435217E
:103E4000FC011382128288EE93E0A0E0B0E084834C
:103E50009583A683B78386EC92E0918380837587F0
:103E6000648757874687318B208B138B028BF58AAB
:103E7000E48AD78AC68AB18EA08E938E828E8F8571
:103E8000848F8889858F8989868F8A89878F8B8996
:103E900080A3ECE00C945121CF92DF92EF92FF923D
:103EA000CF93DF93EC016A017B01411581EE580746
:103EB00061057105F9F0EC89FD8981E090E008A0C9
:103EC00002C0880F991F0A94E2F7808360E079E0CE
:103ED0008DE390E0A70196010E94EE202150310968
:103EE000410951095695479537952795211580E148
:103EF000380798F0EC89FD89108260E874E88EE15B
:103F000090E0A70196010E94EE202150310941095D
:103F100051095695479537952795E889F989308352
:103F2000EA89FB89208319A2EE89FF89408181E01B
:103F300090E09C010C8C02C0220F331F0A94E2F720
:103F4000422B4083EE89FF8940819C010D8C02C089
:103F5000220F331F0A94E2F7422B4083EE89FF8938
:103F600040819C010E8C02C0220F331F0A94E2F79D
:103F7000422B4083EE89FF8920810F8C02C0880F7D
:103F8000991F0A94E2F7809582238083DF91CF9175
:103F9000FF90EF90DF90CF900895BF92CF92DF9285
:103FA000EF92FF92CF93DF93EC016A017B01B22E77
:103FB000411581EE580761057105F9F0EC89FD891D
:103FC00081E090E008A002C0880F991F0A94E2F7F0
:103FD000808360E079E08DE390E0A70196010E9484
:103FE000EE202150310941095109569547953795E1
:103FF0002795211580E1380798F0EC89FD8910821A
:1040000060E874E88EE190E0A70196010E94EE203E
:104010002150310941095109569547953795279502
:10402000E889F9893083EA89FB892083E88DF98D55
:10403000B082EE89FF89408181E090E09C010C8C88
:1040400002C0220F331F0A94E2F7422B4083EE890D
:10405000FF8940819C010D8C02C0220F331F0A94FE
:10406000E2F7422B4083EE89FF8940819C010E8C50
:1040700002C0220F331F0A94E2F7422B4083EE89DD
:10408000FF8920810F8C02C0880F991F0A94E2F7E4
:10409000809582238083DF91CF91FF90EF90DF9016
:1040A000CF90BF9008958F929F92AF92BF92CF9280
:1040B000DF92EF92FF920F931F9381E08F9385E041
:1040C0008F9387E08F9383E08F9384E08F93E6EC68
:1040D0008E2E912CF2ECAF2EB12CA1ECCA2ED12C4D
:1040E000B0ECEB2EF12C04EC10E025EC30E044E3D6
:1040F00054E068E774E082E194E00E941A1F0F9098
:104100000F900F900F900F901F910F91FF90EF90D5
:10411000DF90CF90BF90AF909F908F9008950E94B6
:10412000CA1B0E945E12C6EDDEE10E945016209767
:10413000E1F30E94D61EF9CFA29FB001B39FC00148
:10414000A39F700D811D1124911DB29F700D811DC3
:104150001124911D08950E949C20A59F900DB49F4D
:10416000900DA49F800D911D11240895B7FF0C940C
:10417000AB200E94AB20821B930B0895DB018F9331
:104180009F930E94AB20BF91AF91A29F800D911D84
:10419000A39F900DB29F900D11240895991B79E073
:1041A00004C0991F961708F0961B881F7A95C9F7C7
:1041B00080950895AA1BBB1B51E107C0AA1FBB1F16
:1041C000A617B70710F0A61BB70B881F991F5A95A3
:1041D000A9F780959095BC01CD010895A1E21A2E12
:1041E000AA1BBB1BFD010DC0AA1FBB1FEE1FFF1F9B
:1041F000A217B307E407F50720F0A21BB30BE40BEB
:10420000F50B661F771F881F991F1A9469F7609531
:104210007095809590959B01AC01BD01CF010895EB
:10422000052E97FB1EF400940E94272157FD07D00E
:104230000E94EE2007FC03D04EF40C9427215095E9
:104240004095309521953F4F4F4F5F4F0895909582
:104250008095709561957F4F8F4F9F4F08952F9256
:104260003F924F925F926F927F928F929F92AF9206
:10427000BF92CF92DF92EF92FF920F931F93CF9353
:10428000DF93CDB7DEB7CA1BDB0B0FB6F894DEBFEA
:104290000FBECDBF09942A88398848885F846E8410
:1042A0007D848C849B84AA84B984C884DF80EE805A
:1042B000FD800C811B81AA81B981CE0FD11D0FB663
:1042C000F894DEBF0FBECDBFED010895EE0FFF1FC6
:1042D0000590F491E02D0994FB01DC0102C00190EE
:1042E0000D9241505040D8F70895F999FECF92BDF4
:1042F00081BDF89A992780B50895262FF999FECFA8
:104300001FBA92BD81BD20BD0FB6F894FA9AF99AF2
:0A4310000FBE01960895F894FFCF48
:10431A000000BC04200008409CFF00881300020033
:10432A000200020002000200020002000200020073
:10433A000200020002000200020002000200200144
:10434A002201260221022703230326042605260525
:10435A002B0624072507280729072A802500000598
:10436A00400AA1204EA50020244EA52C2330C012BD
:10437A0000001A400AA1204EA5001B1E27522C231A
:10438A00308025000005400AA1204EA50020244EB9
:10439A00A52C2330004B000006400AD0009D49009E
:1043AA007B289D492C233000E1000005400A450185
:1043BA00D7DC03B81E0EBF00232E48E801008A404E
:1043CA000A6001555502AD1E20000023C801545849
:1043DA002074696D656F7574210057616974696E1F
:1043EA00672062696E640A00476F7420706B740AF2
:1043FA00006461746120676F6F640A007363616EA1
:10440A006E6572206D6F6465004F70656E4C525315
:10441A006E67205258207374617274696E67200047
:10442A00206F6E20485720005361766564206269C8
:10443A006E64206461746120746F20454550524F48
:10444A004D0A004920616D20736C61766500456EE6
:10445A00746572696E67206E6F726D616C206D6F24
:10446A00646500454550524F4D2064617461206E69
:10447A006F742076616C6964206F722062696E6461
:10448A00206A756D70706572207365742C20666F72
:10449A007263696E672062696E640A005258206806
:1044AA00616E6700B200F4014C0300070B0C101197
:1044BA001500091203130E0F00010200000010007C
:1044CA0000000800200000010000020000000100B6
:1044DA000002000000005E1EE01C041E311E161EB3
:0244EA00531E5F
:107E00000F92CDB7DEB7112484B714BE81FFF1D035
:107E100082E08093C00088E18093C10086E0809377
:107E2000C20080E18093C4008EE0CDD088249924E4
:107E3000CC24C394F5E0DF2EE1E1EE2E73E0F72EC3
:107E4000B6D0082F813479F4B2D08983C2D0898129
:107E5000823811F481E005C0813811F485E001C059
:107E600083E09ED09AC0823411F484E103C085344B
:107E700019F485E0B6D091C0853561F498D0082F0B
:107E800010E095D090E0982E8824802A912A880CC2
:107E9000991C82C0863521F484E0A3D080E0E1CF34
:107EA000843609F04CC083D082D0A82E80D0B82E62
:107EB00000E011E07CD0F80181938F01AE16D1F77C
:107EC00088D0FB2DF53489F4E0E0F1E00BC0F9999E
:107ED000FECF92BC81BC0894811C911C819180BD15
:107EE000FA9AF99AEA1598F358C08B2D863409F05E
:107EF00054C0F401F7BEE89507B600FCFDCFF401CD
:107F0000A0E0B1E02C9130E011968C91119790E0B7
:107F1000982F8827822B932B12960C01C7BEE895C9
:107F20001124329681E0A038B80761F7F401D7BE7A
:107F3000E89507B600FCFDCFE7BEE8952EC0843774
:107F4000F1F435D034D0182F32D0B82E42D0FB2DDA
:107F5000F63421F4F40105914F010CC0FB2DF534EA
:107F600049F4F999FECF92BC81BC0894811C911C04
:107F7000F89A00B5802F14D0115049F70EC08537FC
:107F800039F427D08EE10CD085E90AD08FE069CF93
:107F9000813511F488E017D01CD080E101D050CF9A
:107FA0009091C00095FFFCCF8093C600089580910A
:107FB000C00087FFFCCF8091C00084FD01C0A89560
:107FC0008091C6000895E0E6F0E098E19083808318
:107FD0000895EDDF803219F088E0F5DFFFCF84E10E
:107FE000DFCF1F93182FE3DF1150E9F7F2DF1F9166
:0E7FF0000895282E80E0E7DFEE27FF27099492
:027FFE0001057B
:0400000300007E007B
:00000001FF
